:1000000080313E28080008007E14803120007F08DF
:10001000F6002100111C13282000111C13288B311D
:100020007B23803139282100911D1D282000911D3E
:100030001D2884314D24803139282100921D272824
:100040002000921D27288B31682380313928210018
:10005000911E31282000911E31288C316B24803173
:1000600039282100111E39282000111E39288C3111
:100070002E2476082000FF007E10090080314028E1
:10008000F701F801F901FA01FB01E03084000030CA
:1000900085000F308B317523803120308400013092
:1000A00085002E308B3175238031A03084000130E3
:1000B000850040308B317523803120308400023040
:1000C000850028308B3175238031C73084008B3018
:1000D00085004E3086000130870018308B316F2349
:1000E0007E1020008631742E0034C13481344034B7
:1000F0000134C034803441340134C034803441345C
:100100000034C134813440340134C034803441344B
:100110000034C134813440340034C134813440343B
:100120000134C034803441340134C034803441342B
:100130000034C134813440340034C134813440341B
:100140000134C034803441340034C134813440340B
:100150000134C034803441340134C03480344134FB
:100160000034C134813440340134C03480344134EB
:100170000034C134813440340034C13481344034DB
:100180000134C034803441340034C13481344034CB
:100190000134C034803441340134C03480344134BB
:1001A0000034C134813440340034C13481344034AB
:1001B0000134C034803441340134C034803441349B
:1001C0000034C134813440340134C034803441348B
:1001D0000034C134813440340034C134813440347B
:1001E0000134C034803441340134C034803441346B
:1001F0000034C134813440340034C134813440345B
:100200000134C034803441340034C134813440344A
:100210000134C034803441340134C034803441343A
:100220000034C134813440340034C134813440342A
:100230000134C034803441340134C034803441341A
:100240000034C134813440340134C034803441340A
:100250000034C134813440340034C13481344034FA
:100260000134C034803441340034C13481344034EA
:100270000134C034803441340134C03480344134DA
:100280000034C134813440340134C03480344134CA
:100290000034C134813440340034C13481344034BA
:1002A0000134C034803441340134C03480344134AA
:1002B0000034C134813440340034C134813440349A
:1002C0000134C034803441340034C134813440348A
:1002D0000134C034803441340134C034803441347A
:1002E0000034C134813440340034C034C13401346A
:1002F000C33403340234C234C63406340734C7343A
:100300000534C534C4340434CC340C340D34CD3409
:100310000F34CF34CE340E340A34CA34CB340B34D9
:10032000C93409340834C834D83418341934D934A9
:100330001B34DB34DA341A341E34DE34DF341F3439
:10034000DD341D341C34DC341434D434D534153449
:10035000D73417341634D634D23412341334D33459
:100360001134D134D0341034F03430343134F134E9
:100370003334F334F23432343634F634F734373439
:10038000F53435343434F4343C34FC34FD343D3409
:10039000FF343F343E34FE34FA343A343B34FB34D9
:1003A0003934F934F83438342834E834E934293429
:1003B000EB342B342A34EA34EE342E342F34EF3439
:1003C0002D34ED34EC342C34E43424342534E53449
:1003D0002734E734E63426342234E234E334233459
:1003E000E13421342034E034A03460346134A13469
:1003F0006334A334A23462346634A634A734673439
:10040000A53465346434A4346C34AC34AD346D3408
:10041000AF346F346E34AE34AA346A346B34AB34D8
:100420006934A934A83468347834B834B9347934A8
:10043000BB347B347A34BA34BE347E347F34BF3438
:100440007D34BD34BC347C34B43474347534B53448
:100450007734B734B63476347234B234B334733458
:10046000B13471347034B0345034903491345134E8
:100470009334533452349234963456345734973438
:1004800055349534943454349C345C345D349D3408
:100490005F349F349E345E345A349A349B345B34D8
:1004A0009934593458349834883448344934893428
:1004B0004B348B348A344A344E348E348F344F3438
:1004C0008D344D344C348C34443484348534453448
:1004D0008734473446348634823442344334833458
:1004E00041348134803440342000BB00BD01F830F9
:1004F0003B02031C7F2A1230B6003608BD003D08BF
:100500000319312C4B2C2E0303198A2A02302E0694
:10051000031D922A3108320403199D2A0030320249
:100520004130992A3108320403199D2A00303202E1
:10053000213003193102031CA12A1330B6003608FA
:10054000BD003D08031D4B2C3B08B6003408860057
:100550008701360881002E08B600340A860087011C
:10056000360881002F08FF3EB600FF30303DB7004F
:100570003708B8003408023E860087013808810039
:100580002F08FF3EB6003408033E86008701360878
:1005900081003208B6003408043E86008701360820
:1005A00081003108B6003408053E86008701360810
:1005B00081000530B60034081E3E860087013608EB
:1005C000810034088E318926823120002E030319E0
:1005D000ED2A02302E06031D0A2B3208B70031081F
:1005E000B600B736B60CB736B60CB736B60C36080A
:1005F000B8003808BC0007303105B60000303205BD
:10060000B7003608370403190E2B0130B600360840
:10061000BC070E2B3135B6003608BC003C08023E44
:10062000242C05302E06031D2F2B330886000130A5
:1006300087000103031D212B0030B900FF30BA00F1
:100640002F2B33088600013087000108031D2B2B58
:10065000B901BA012F2B1030B6003608BD003103A6
:1006600032040319372B1330B6003608BD003D089D
:10067000031D4B2C3B08B600340886008701360862
:1006800081002E08B600340A8600870136088100F2
:100690002F08FF3EB600FF30303DB7003708B800E6
:1006A0003408023E86008701380881002F08FF3E8B
:1006B000B6003408033E8600870136088100053005
:1006C0002E06031D672B3930A00000306B2B200055
:1006D0003308A0000130A1003408043EB6003608FB
:1006E000A2000130A3000030A4008D31EC2582313E
:1006F00005302000172C0F302E0631083204031964
:10070000882B00303202413003193102031C8C2B3C
:100710001330B6003608BD003D08031D4B2C0F30CA
:100720002E06031DB02B3208B7003108B600B736CD
:10073000B60CB736B60CB736B60C3608B800380863
:10074000BC0007303105B60000303205B70036086E
:1007500037040319B42B0130B6003608BC07B42B9C
:100760003135B6003608BC003B08B60034088600B8
:100770008701360881002E08B600340A86008701FA
:10078000360881002F08FF3EB600FF30303DB7002D
:100790003708B8003408023E860087013808810017
:1007A0002F08FF3EB6003408033E86008701360856
:1007B00081003208B6003408043E860087013608FE
:1007C00081003108B6003408053E860087013608EE
:1007D00081003C08B6003408063E860087013608D2
:1007E00081000F302E06031D032C3408073EB6008F
:1007F0003608A0003208A2003108A10033088F316A
:100800009E278231142C20003308A0000130A10063
:100810003408073EB6003608A2003208A4003108AA
:10082000A3008D31EC25823120003C08063EB60045
:1008300034081E3E860087013608810034088E3158
:100840008926823105302000B60035081E3E86001C
:100850008701360881004B2C0A30B6003608BD00EF
:100860004B2C2E08013A0319832A033A0319832AD1
:10087000013A0319832A073A0319832A013A031913
:10088000112B033A0319112B093A03197B2B1F3A39
:1008900003197B2B2C2C3D0808002000911124000B
:1008A000951F8A2D95132100ED017808023E8600E0
:1008B000013087000108860087018101810AF80163
:1008C0000800E21808006108F2007208F8006108E8
:1008D0008600013087000108F2007208EE0061080E
:1008E0008600013087000130413FF9000430F200FA
:1008F0007208E10761084E3A031D822C4A30F2006B
:100900007208E1006210610860060319E214240015
:1009100016140230F20072082100ED0008002400D5
:1009200096140230F20072082100ED000800240045
:10093000161FA32C0130F20072082100E4070430D6
:100940008B31F82308007B08F3007A08F200F336B5
:10095000F20C7208240091007A1CB42C0B30F200C7
:1009600072082100ED0008000330F2007208210037
:10097000ED0008002400161FC62C0130F20072089A
:100980002100E40704308B31F823080096147B081B
:10099000F3007A08F2007308F200F30106307205E2
:1009A000F40000307305F500F0307404FA000030F4
:1009B0007504FB007A142100E501E50A0230F2001B
:1009C0007208ED00080065030319FC2C7908860005
:1009D00001308700403FFA00413FFB007908860064
:1009E000013087000130433FE7007908860001307D
:1009F00087000130423FE6007A08240091007A1C0B
:100A0000072D0530F20072082100ED0008000330C8
:100A1000F20072082100ED0008002400161F1B2DB3
:100A20000130F20072082100E4072400161305309B
:100A30008B31F823080001302100E602660A031D0D
:100A4000352D0530F2007208F9070130EE02031D62
:100A50002D2D00308B31F82308002400961402302D
:100A6000F20072082100ED00080067088600870187
:100A70000108240091000130F20072082100E7070C
:100A800008002400161F4F2D0130F20072082100CB
:100A9000E40704308B31F823240016130800961560
:100AA0000830F20072082100ED0008000830F20062
:100AB0007208ED0024009615080024001108F200C9
:100AC0002100670886008701720881000130F2006A
:100AD0007208E7070130E6020319762D240096120A
:100AE0000630F20072082100ED007A2D24009616DF
:100AF0008B31922324001616080000308B31F82326
:100B000008000130F20072082100E40706308B3142
:100B1000F823080021006D0884000C30040203183B
:100B2000812D88310435003E820008002000B90084
:100B3000B801300886008701390884008501000863
:100B400001060319A52D0630502E30088E31E326FC
:100B50008531013A0319AF2D07302000502E2000B7
:100B6000300A86008701811FC32D3008023E8600AF
:100B700087010108B400310886000130870034087D
:100B800081000D30502E300A86008701390A84001A
:100B90008501000801060319542E0E30502E33082B
:100BA000B5003208B400B536B40CB536B40CB53661
:100BB000B40C3408B6003608B70007303205B4006C
:100BC00000303305B500340835040319EB2D01302E
:100BD000B4003408B7073008023E860087010108D8
:100BE0003706031D0E2E3108B4003408A000330868
:100BF000A2003208A1003008033E8E313A2685312A
:100C0000712E20003235B4003408B7003008023E9F
:100C100086008701010837060319102E0F30502E69
:100C20003108B4003408A0003308A2003208A10043
:100C30003008033E8D3158258531712E2000300853
:100C4000023E860087013908023E840085010008C3
:100C50000106031D4F2E3008033E86008701390828
:100C6000033E8400850100080106031D4F2E300855
:100C7000043E860087013908043E8400850100088F
:100C80000106031D4F2E3008053E860087013908F6
:100C9000053E84008501000801060319712E1030FD
:100CA000B4003408B800712E300A860087010108AC
:100CB000013A0319CF2D033A0319CF2D013A031935
:100CC000012E073A0319012E013A03191E2E033A89
:100CD00003191E2E093A03191E2E1F3A03191E2E40
:100CE000712E200038080800220061082000EB0067
:100CF000220060082000EA0022005F082000E900CE
:100D000022005E082000E800220065082000EF00B5
:100D1000220064082000EE00220063082000ED009D
:100D2000220062082000EC002100A0012000E70161
:100D30002100A1014E308600013087005730840029
:100D40000030850008302000D20016001A00D20BB7
:100D5000A52E56308600013087005F3084000030B9
:100D600085000830D20016001A00D20BB32E8B314A
:100D7000B52386318C318D2486318B170B170030CB
:100D8000803103208631C52EA101A2302000D2007F
:100D90005208BE00210020082000D3005308BF00E5
:100DA00021002108683E8600870101082000D40048
:100DB0005408C000210021086C3E8600870101080C
:100DC0002000D5005508C100210021355F3E860076
:100DD0008701403F2000C200413FC3002100213570
:100DE000573E86008701403F2000C400413FC500B8
:100DF000C030D6005608C600C1308D31A2258631DC
:100E0000A2302000D2005208BE002100200820009D
:100E1000D3005308BF0021002108683E86008701E7
:100E200001082000D4005408C000210021086C3EB5
:100E30008600870101082000D5005508C100210067
:100E400021355F3E86008701403F2000C200413FC0
:100E5000C30021002135573E86008701403F200016
:100E6000C400413FC500C030D6005608C600C1309E
:100E70008F31402786310330210021060319C42E0B
:100E800001302000D20052082100A107C52E200009
:100E9000AF01AF0AB201B301B001B101AD01AE01C2
:100EA0002A08860087018101B001B10100303102BA
:100EB0001430031930020318A52F8B31A323873177
:100EC00020002108AE002008AD0021009112690821
:100ED000203E86000130870001082000AB00320868
:100EE0002907AC002C08860087012B0881000130FF
:100EF0002100E802911601302000AB002B082100F0
:100F0000E9071E3069020318E90101302000B20729
:100F10000030B33D8B31A323873120002108AE0080
:100F20002008AD0027083306031D982F2608320637
:100F30000319A52F0130B0070030B13D0030310258
:100F4000143003193002031C5D2F27083306031DDC
:100F5000AB2F26083206031DB92F2808860087010B
:100F60003208C03F3308C13F2A088600870181014B
:100F7000C12F0530AB002A08860087012B088100AD
:100F8000AF012F0808002000A801A80A2100E801ED
:100F9000E901F7012000A901AA0123082A02031D83
:100FA000D32F220829020318E52F29082507A700B7
:100FB00027088600870101088C31B0248731013071
:100FC0002000A9070030AA3DCD2F24088600870104
:100FD0002208C03F2308C13F2608860087018101FF
:100FE0002808080005302800970005309600950174
:100FF0002000931008002100E801E901F701080032
:101000008431612C84318F2C8431E32C85310D2D7A
:1010100085317D2D8531412D8531562D85317D2DB3
:1010200085315D2D8531812D8431972C8431BA2C09
:1016D00008006A30210099009A0198010800FE0074
:1016E00012001E00FE0B702B0034640080010131DB
:1016F000890B762B0034200011107D0897007C08A0
:101700009600080089302000980010309900803041
:10171000970096011708FD001608FC001110210023
:10172000111408000530F0007008F907013021009D
:10173000EE02031DA02B0430F0007008ED0008003D
:10174000ED01ED0A08002100911268082000A200B6
:10175000A3012208A4002308A5002100911620005F
:101760002508A1002408A00008008B3169238B31D3
:101770008D3101258B318731F2278B318B318223DB
:101780008B318C3112248B318B31DF2308001034E4
:101790000034103400340A3400340A340034013484
:1017A0000034013400340134003401340034013495
:1017B000013401340134013402340334043421008F
:1017C00091121112483023009F0090309D00263066
:1017D0009E0068309B009C012100EB01EC010F3062
:1017E0002000A00020082100EF00EA019116080067
:1017F000F100240016157808023E860001308700AB
:10180000010803190F2C7108F0007808023E8600C9
:1018100001308700010886008701700881002100DF
:10182000ED0108004A302000A00020082100E1005E
:101830004A302000A00020082100E000E2146210DD
:10184000E40180302400940028309500970109308D
:101850009200200091112100911508000F30210005
:101860006F020318492C6C082F3E86000130870058
:10187000010823009A000130F00070082100EC07F5
:101880000F306C020318EC010130F0007008EF0714
:101890000800111208002000A3002308A100043052
:1018A000A136890B502C2108A2002208A30023088E
:1018B0000F39A1002108A3000F08F0398F000F088D
:1018C00023048F002008031D0F1603190F128F1217
:1018D0000F170F13080023001908F0007008F1001B
:1018E000200091120F307702031808007108F000F1
:1018F0007708203E860001308700700881000130A3
:10190000F0007008F7070F3077020318F701013075
:10191000F00070082100E807080020008F01210076
:101920008F0120008F171430A8007930A700A70B73
:10193000972CA80B972C003232308C31D8248C3164
:1019400028308C31D8248C310C308C31D8248C3117
:1019500001308C31D8248C3106308C31D8240800E9
:101960002000A10021006F080319B22C111ABD2C10
:101970002000210823009A00D52C111220002108F4
:10198000A00021006B082F3E860001308700200058
:10199000200881000130A00020082100EB070F3053
:1019A0006B020318EB010130EF0221001116080051
:1019B0002000A6000730A5007D30A400A40BDE2C7B
:1019C000A50BDE2C2000A00126088C314B248C3185
:1019D00020002608A4000330A435FF3E031DEC2C94
:1019E0002435A5002508A600F930A4000000A40BAA
:1019F000F62C003200002000A00126088C314B2478
:101A0000080022008C01FF3021008C0001302300EF
:101A10008C0022008D01013021008D0023008D01FA
:101A200024008D01183022008E00FB3021008E0032
:101A300022008F0121008F0123008F0122009001DD
:101A40000F3021009000230090012400900121001C
:101A5000951722009D0108002000BA00BD0136083C
:101A6000A7003508A6003B30B7003708A8003408A7
:101A7000B8003808A9003D30B9003908AA003A0872
:101A8000873147278D31003A031D492D20003D083D
:101A9000080020003B08B7003708B4073B08B50230
:101AA0003C08B63B35083604031D2F2D3D080800C1
:101AB0002000A900AA01AB01A8012808A300A401E5
:101AC00022082402031D662D2108230203180800A2
:101AD0002A082907A3002308860087010108A4001B
:101AE000A5012408A500A4012B352007A70027087D
:101AF0008600013087002408C03F2508C13F2A081E
:101B0000013E2907A3002308860087010108A400DD
:101B1000A5012B352007A600260886000130870086
:101B2000240881044131250881040130A3002308E1
:101B3000AB070230A3002308AA070130A300230843
:101B4000A8075D2D2000D000D1014108C70047083B
:101B5000AE004308B0004208AF004508B200440898
:101B6000B1004608C8004808B3005008C900490839
:101B7000B4003E08CA004A08B50040088231742209
:101B80008D312000CB004B08D1005108031D080007
:101B900050081E3E860087010108033ECC0000303D
:101BA00003180130CD003F088731FB278D3120001D
:101BB0004D08A3004C08A2004E30C7004708A400FF
:101BC0005008C8004808A5005130C9004908A600BF
:101BD0003F088731C32708002000AC01AD01AB01ED
:101BE0002B08A500A60124082602031DF92D2308B1
:101BF0002502031808002C08A500A601A535A60D8E
:101C00002508200786002608213D8700403FA700C1
:101C1000413FA8002808A9002D082207AA002A0889
:101C200086008701290881000130A5002508AD073D
:101C30002C08A500A601A535A60D250820078600BD
:101C40002608213D87000108A7002D082207A800CB
:101C5000280886008701270881000130A500250893
:101C6000AD070130A5002508AC070130A500250807
:101C7000AB07F02D2000A700A801A901AA01AB0124
:101C8000AD01AE0122082E02031D482E21082D02AF
:101C900003180800AC01AC0AAF0108302F0203188A
:101CA000842E28082707A30023088600870101083F
:101CB0002C05A4002F0A5D2EA436890B5C2E240867
:101CC000A5002A082007A600260886000130870004
:101CD000250881000130AA070030AB3D0310AC0D90
:101CE0000130AD070030AE3D22082E02031D7A2ED2
:101CF00021082D02031808000130A3002308AF07B4
:101D000008302F02031C512E0130A8070030A93DD6
:101D1000422E2000A900FF30A0002008A500FF30BF
:101D2000A0002008A60029081E3E860087010108A1
:101D3000013EA0002008A800A701280827020318D8
:101D4000CD2E27082907A00020088600870101085A
:101D50002606A100A2012108A3002208A40024084D
:101D6000850023088400743084078030853D000896
:101D70002506A0002008A60024088500230884006A
:101D8000743084078130853D0008A0002008A5003C
:101D90000130A0002008A7079D2E2608A0002808D3
:101DA0002907A10021088600870120088100250855
:101DB000A0002808013E2907A1002108860087010C
:101DC0002008810008002000A900FF30A0002008A2
:101DD000A500FF30A0002008A60029081E3E8600AE
:101DE00087010108013EA0002008A800A7012808DB
:101DF00027020318272F27082907A000200886009C
:101E0000870101082606A100A2012108A3002208DB
:101E1000A4002408850023088400743084078030DF
:101E2000853D00082506A0002008A600240885009E
:101E300023088400743084078130853D0008A000A9
:101E40002008A5000130A0002008A707F72E2808C9
:101E50002907A00020088600870101082606031D27
:101E60003E2F2808013E2907A00020088600870190
:101E700001082506031D3E2F013008000030080030
:101E80002000CA00CB014008031908003E08C70023
:101E90004708B4000230B5000030B6003F088D316D
:101EA0002C258F312000C8004808CB004B08031DAB
:101EB00008003E0A86008701811F6B2F0330CC008B
:101EC0000030CD000230C7003E081E3E860087016C
:101ED00047088100762F3E081E3E860087010108D4
:101EE000013ECC00003003180130CD003E08023E18
:101EF000C7004708B4004D08B6004C08B5003F08BD
:101F00008D312C258F312000C8004808CB004B08AC
:101F1000031D08003E08C7004708B0004608C80077
:101F20004808B1004508B3004408B2004A088531AA
:101F300096252000C9004908CB0008002000A70012
:101F4000A901AA012208A4002108A300A436A30C19
:101F5000A436A30CA436A30C2308A5002508A800CA
:101F600007302105A30000302205A4002308240423
:101F70000319BE2F0130A3002308A807AB012808CE
:101F80002B02031808002B082007A3002308860053
:101F900087018101AC0108302C020318FB2F2908AE
:101FA0002707A30023088600013087000108A4004A
:101FB0002C0ADB2FA435890BDA2F2408A5002B0867
:101FC0002007A60026088600870125088104013025
:101FD000A9070030AA3D22082A02031DF12F21087B
:101FE0002902031808000130A3002308AC070830B9
:101FF0002C02031CCF2F0130A3002308AB07BF2FF7
:020000040001F9
:04000E00E4C1FFDC6E
:00000001FF
